:1000000009C025C00DC00CC00BC00AC009C008C083
:1000100007C006C011241FBECFE9CDBF50D0ACC071
:10002000EFCF86B1806C86B93699FECF84B185B1A9
:10003000379890E06EE170E08DD09C0128513C4FE4
:10004000C9010895EEDFC09A68D0C09808951F9244
:100050000F920FB60F9211242F933F934F935F93FC
:100060006F937F938F939F93AF93BF93EF93FF9380
:100070008FEF9DEEA2E081509040A040E1F700C0DC
:100080000000B19902C0C39ADDDF8FEF9BE7A2E9C0
:1000900081509040A040E1F700C00000FF91EF9137
:1000A000BF91AF919F918F917F916F915F914F9190
:1000B0003F912F910F900FBE0F901F901895F894BD
:1000C00087B3896087BBC19A8BB780648BBF85B7C4
:1000D000826085BF17B887B1826687B97894C09867
:1000E000C39A8FE79BEB0197F1F700C00000C3981C
:1000F0008FEF97E9AAE381509040A040E1F700C05C
:100100000000EDCF07C0EFE5F9E03197F1F700C04F
:10011000000081508823B9F7089507C0EFE5F9E0A2
:100120003197F1F700C0000001970097B9F70895E3
:1001300005C093E09A95F1F7000081508823C9F734
:10014000089505C023E02A95F1F700000197009774
:10015000C9F708955527002480FF02C0060E571FD7
:10016000660F771F6115710521F0969587950097A9
:0C01700099F7952F802D0895F894FFCF8B
:00000001FF
